:100000000C941E060C94C3270C94F0270C944606FF
:100010000C9446060C94E9120C9446060C94460681
:100020000C9446060C9446060C9446060C94460620
:100030000C9446060C9446060C9446060C94460610
:100040000C941D280C9446060C940B2C0C944E2CEE
:100050000C9446060C9446060C9446060C944606F0
:100060000C9446060C9446065318B5189418971825
:100070009A189D18A018A318A618B518AF18E71954
:10008000E919E919E719E919E919E919E919E91962
:10009000E919E919E919E919E919E919E919E91950
:1000A0006D19E919E919E919E919E919DE18E919C8
:1000B000E919E919E919E919E919E919E919E91930
:1000C000E919E919E919E919E919E9197919791900
:1000D0007919791979197919791979197919E91920
:1000E000E919E919E919E919E919DE1878197819EE
:1000F00078197819E91986198C19921998199E1985
:10010000A419AA19B019BA19C419CE19D8191F19E6
:10011000E118E919E919E919E9196D19E919E91954
:10012000E919E919E919E919E919E91977197719A3
:1001300077197719E91986198C19921998199E1946
:10014000A419AA19B019BA19C419CE19D8191F19A6
:10015000E118E919E919E919E9196D191C1A1C1AAC
:100160001C1A1C1A1C1A1C1A1C1A1C1A1C1A1C1ADF
:100170001C1A1C1A1C1A331B331B331B331B331B57
:10018000331B611A6B1A751A7F1ADD1AE71AF61AF1
:10019000071B8F1CA41CB01CB91CC81CED1CF61C32
:1001A0003F1D081D522058205E2065207320952099
:1001B000B320456E746572206D656E752E2E2E000F
:1001C000546F67676C6564206D6963726F50504D42
:1001D00000546F67676C656420696E76657274653C
:1001E000642050504D2100546F67676C6564205443
:1001F00058206D7574696E672100546F67676C6570
:10020000642074656C656D65747279210050726F3D
:10021000746F636F6C206572726F72207769746897
:100220002052580054696D656F7574207768656E4B
:1002300020636F6E6E656374696E6720746F205201
:100240005800507265737320616E79206B65792058
:10025000746F2063616E63656C00436F6E6E6563DF
:1002600074696E6720746F2052582C20706F776508
:100270007220757020746865205258202877697440
:10028000682062696E6420706C7567206966206EF4
:100290006F74207573696E6720616C776179732064
:1002A00062696E642900546F67676C656420276912
:1002B0006D6D656469617465206F75747075742700
:1002C00000546F67676C65642027736C61766520E6
:1002D0006D6F64652700546F67676C6564202761E4
:1002E0006C776179732062696E642700546F676769
:1002F0006C65642050504D206368616E6E656C20A3
:100300006C696D69740053657420525353492069B8
:100310006E6A656374696F6E206368616E6E656C8A
:100320002028303D3D64697361626C652900536526
:10033000742050504D206D696E696D756D20737914
:100340006E630053657420626561636F6E20696E31
:1003500074657276616C0053657420626561636FC9
:100360006E2064656C617900536574206265616319
:100370006F6E206672657175656E637920696E2097
:10038000487A3A20303D64697361626C652C205074
:10039000783D504D52206368616E6E656C20782CFC
:1003A0002046783D465253206368616E6E656C202E
:1003B00078005365742050574D2073746F7020641B
:1003C000656C61792028302064697361626C6564B2
:1003D0002C20312D323535203D3D20302E317320FB
:1003E0002D2035306D696E29005365742050504DB5
:1003F0002073746F702064656C61792028302064EC
:10040000697361626C65642C20312D323535203D75
:100410003D20302E3173202D2035306D696E29003E
:10042000536574206661696C736166652064656CF0
:1004300061792028302064697361626C65642C20C6
:10044000312D323535203D3D20302E3173202D2089
:1004500035306D696E29002A2A2A2A2A2A2A2A2A50
:100460002A2A2A2A2A2A2A2A2A2A2A2A2A2A2A2AEC
:100470002A2A2A2A0052582041636B6564202D20C5
:1004800072657665727420737563636573736675E0
:100490006C21002A2A2A2A2A2A2A2A2A2A2A2A2AAD
:1004A0002A2A2A2A2A2A2A2A2A2A2A2A2A2A2A2AAC
:1004B000002A2A2A2A2A2A2A2A2A2A2A2A2A2A2AC6
:1004C0002A2A2A2A2A2A2A2A2A2A2A2A2A2A00528E
:1004D000582041636B6564202D20757064617465DC
:1004E000207375636365737366756C21002A2A2A0D
:1004F0002A2A2A2A2A2A2A2A2A2A2A2A2A2A2A2A5C
:100500002A2A2A2A2A2A2A2A2A2A0056616C696457
:100510002063686F69636573206172653A205B319F
:100520005D2D5B31365D20286368616E6E656C20E1
:10053000312D31362900536574206F7574707574D0
:1005400020666F7220706F727420005B585D2061AE
:10055000626F7274206368616E67657320616E6498
:10056000206578697420525820636F6E6669670051
:100570005B535D20736176652073657474696E6783
:100580007320746F205258005B525D20726576654F
:1005900072742052582073657474696E6773207486
:1005A0006F2064656661756C747300557365206EA9
:1005B000756D62657273205B312D445D20746F2010
:1005C0006564697420706F727473205B452D515D92
:1005D00020666F722073657474696E677300202DD6
:1005E00020726563656976657220636F6E66696700
:1005F000757261746F722C20727820737720000AF4
:100600000A6F70656E4C52536E67200053657420FC
:1006100073657269616C2062617564726174653AB8
:10062000200056616C69642063686F696365733A82
:100630002031202D20342B34202F2032202D203823
:10064000202F2033202D20382B34202F2034202D14
:10065000203132202F2035202D2031322B34202FF5
:100660002036202D20313600536574204368616E9A
:100670006E656C20636F6E6669673A20005365741F
:100680002044617461726174652028302D32293AEA
:10069000200053657420486F70206368616E6E653A
:1006A0006C7320286D61782032342C207365706162
:1006B000726174656420627920636F6D6D61732966
:1006C0002076616C69642076616C75657320312DCC
:1006D0003235353A2000536574206368616E6E656B
:1006E0006C2073706163696E6720287831306B48C5
:1006F0007A293A200053657420524620706F77653E
:10070000722028302D37293A200053657420524634
:10071000206D6167696320286865782920652E67E8
:100720002E20307844454144463030443A2000532E
:1007300065742062617365206672657175656E63AC
:10074000792028696E20487A293A20005B5A5D207A
:10075000656E746572207265636569766572206383
:100760006F6E66696775726174696F6E2075746902
:100770006C79005B465D20646973706C61792061FF
:10078000637475616C206672657175656E63696509
:10079000732075736564005B525D2063616C6375E3
:1007A0006C6174652072616E646F6D206B65792079
:1007B000616E6420686F70206C697374005B495DC2
:1007C000207265696E697469616C697A6520736508
:1007D0007474696E677320746F20736B65746368DB
:1007E0002064656661756C7473005B585D2072658A
:1007F00076657274206368616E67657320616E64EC
:100800002065786974206D656E75005B535D20739B
:100810006176652073657474696E677320746F20E8
:10082000454550524F4D20616E64206578697420B3
:100830006D656E7500557365206E756D62657273BA
:10084000205B302D395D20746F20656469742070E1
:100850006172616D657465727300202D2053797328
:1008600074656D20636F6E66696775726174696F18
:100870006E000A0A6F70656E4C52536E672000510D
:1008800029204F7574707574206265666F726520DB
:100890006C696E6B20283D465329203A2000502970
:1008A00020536C617665206D6F64652028657870D3
:1008B0006572696D656E74616C293A20004F29205C
:1008C00054696D65642042494E44206174207374FC
:1008D000617274757020203A20004E292050504DCE
:1008E000206F7574707574206C696D69746564200F
:1008F000202020203A200044495341424C454400E6
:100900004D292050504D205253534920746F20637D
:1009100068616E6E656C202020203A20004C2920F2
:1009200050504D206D696E696D756D2073796E63E1
:10093000202875732920203A200044495341424C15
:100940004544004B29204661696C736166652062ED
:100950006561636F6E20696E74762E2028312D32AA
:10096000353573293A20004A29204661696C736144
:10097000666520626561636F6E2064656C617920D5
:1009800028302D323535203D3E20313073202D204A
:100990003135306D696E293A200049292046616958
:1009A0006C7361666520626561636F6E206672714B
:1009B0002E203A200048292050574D2073746F7024
:1009C0002064656C6179202020202020203A2000BE
:1009D00047292050504D2073746F702064656C61FE
:1009E00079202020202020203A200046292046611E
:1009F000696C736166652064656C617920202020D4
:100A00002020203A200050574D206368616E6E65AB
:100A10006C200066756E6374696F6E3A2000292041
:100A2000706F72742000506F776572546F776572C3
:100A300000445446205548462033322D62697420C4
:100A400031306368004F70656E4C52536E67525878
:100A5000206D696E6920342F36636800466C7974A6
:100A6000726F6E2F4F72616E6765525820554846FF
:100A70002038636800525820747970653A20004429
:100A8000697361626C656400487A00203D3D200016
:100A900043616C63756C61746564207061636B6540
:100AA0007420696E74657276616C3A200042292068
:100AB0004D6963726F202868616C66292050504D23
:100AC000202020203A00412920496E766572746505
:100AD000642050504D20696E20202020203A0030A4
:100AE00029204D7574652062757A7A657220286DAB
:100AF0006F73746C79293A003929205365726961E2
:100B00006C2062617564726174653A00736D617224
:100B100074506F7274004672536B79005472616E38
:100B200073706172656E740044697361626C6564B0
:100B30000038292054656C656D657472793A2020FF
:100B40002020202020003729204368616E6E656CCC
:100B500020636F6E6669673A202000362920446161
:100B60007461726174652028302D32293A2020206A
:100B700000352920486F70206368616E6E656C7364
:100B80003A2020202020003429204368616E6E65C1
:100B90006C2073706163696E673A202000332920EE
:100BA000524620706F7765722028302D37293A2001
:100BB0002020003229205246206D616769633A2067
:100BC0002020202020202020003129204261736530
:100BD000206672657175656E63793A202020000089
:100BE00000000700020100000304060000000000EE
:100BF00000000001020408102040800102040810D7
:100C00002001020408102004040404040404040263
:100C10000202020202030303030303000000002395
:100C2000002600290000000000250028002B0000FD
:100C3000000000240027002A00003C2D11241FBEC4
:100C4000CFEFD8E0DEBFCDBF13E0A0E0B1E0E6E833
:100C5000F0E602C005900D92A83CB107D9F716E066
:100C6000A8ECB3E001C01D92AC38B107E1F71CE07D
:100C7000CCE3DCE004C02297FE010E94452ECA337B
:100C8000D107C9F70E94782D0C9441300C940000D4
:100C900080917105813019F482E080937105809113
:100CA0007105833019F484E0809371050895A89547
:100CB0000895DC01ED91FC910190F081E02D099502
:100CC00008952091720530917305382748E0C901D5
:100CD000880F991F37FF06C09C0151E2252750E17C
:100CE000352701C09C01415091F730937305209343
:100CF0007205089588E38093740580E092ECA1E08A
:100D0000B0E08093750590937605A0937705B09336
:100D1000780587E08093810580EC9AECA9E8B6E33A
:100D20008093790590937A05A0937B05B0937C0519
:100D300085E0809382058DEE9EEFADEABEED809357
:100D40007D0590937E05A0937F05B0938005E3E831
:100D5000F5E080E090E0863028F4DC01AE54BC4F32
:100D60002C9101C020E0219301968831910599F7DB
:100D700082E080939B058AE080939C05089580EC37
:100D800097EFAAEBB7E38093B9059093BA05A093C8
:100D9000BB05B093BC0580E090E0A0E0B0E5809397
:100DA000BD059093BE05A093BF05B093C005E1ECCF
:100DB000F5E080E081938F5F8031E1F70895A0E056
:100DC000B0E0E5EEF6E00C940E2ED82F0E947328CA
:100DD0006115710581059105C9F30E94B12E10922C
:100DE0007D0510927E0510927F0510928005C4E06B
:100DF000812C912C54018A94C0907D05D0907E0561
:100E0000E0907F05F0908005FE2CED2CDC2CCC24AE
:100E10000E94AC2EA50194010E94ED2D6C0D7D1D4C
:100E20008E1D9F1D60937D0570937E0580937F05C9
:100E300090938005C15001F7DD2309F450C003E809
:100E400015E0E801A12CB12C62E3C62ED12CE12CD7
:100E5000F12C8881882309F442C0B39419F40E94CC
:100E60007A063DC00E94AC2EA70196010E94ED2D8E
:100E7000E1E0E60FA3E8B5E08A2F801B8A1520F495
:100E80008D918E13F9CFE9CF2091820530E0A0E15A
:100E9000B7E20E94852D9B01AC01AE2FB0E00E940D
:100EA000942D4090790550907A0560907B05709064
:100EB0007C05640D751D861D971D4090B9055090E9
:100EC000BA056090BB057090BC05461657066806CB
:100ED000790618F2E993A39488E1A812BACFCDB7A6
:100EE000DEB7E0E10C942A2E8436910520F4BC0193
:100EF00080E090E017C09C018E3B910528F42A55B4
:100F00003109AAE0B0E00CC0823D910528F4245BD1
:100F10003109A4E6B0E004C02D5C3109A8E5B2E0D7
:100F20000E94852DA4E6B0E09B01AC010E94942DA7
:100F3000089590E08C599F4F0E947407089561E0D6
:100F40008AE00E94202960E08AE00E9459290895E1
:100F5000892B11F061E001C060E08AE00E9459290C
:100F6000089560E089E00E94202961E088E00E9405
:100F7000202961E087E00E94202960E082E00E9451
:100F8000202961E084E00E942029089542E050E099
:100F900068E476E080E00E94A3270895E3E0F0E0B3
:100FA00089E080935700E491E67081E0E63009F033
:100FB00080E00895CF93DF93C82F0E94CE07882347
:100FC00081F0DFB781E080937005F8940E945706A6
:100FD00088E180936000C0936000C1110E945706B1
:100FE000DFBFDF91CF9108958F929F92AF92BF9212
:100FF000CF92DF92EF92FF92CF93FC01C0A5EC2F2E
:10100000E770F0E0E658FC4FA081B0E0C7FF03C0F6
:1010100024E130E002C02FE030E0FC0197A183E141
:10102000989FF0011124E25CFE4F80809180A280A5
:10103000B380A20FB31F20E43FE14DE750E00E94D0
:101040009F2DA50194010E94CB2D8C2F887149F40E
:1010500069017A01E0EDCE0EE7E0DE1EE11CF11C35
:101060001BC0C7FF05C060E47AE88CE29EE004C0C4
:1010700060E07EEE8AEB9BE069017A01F8EBCF0E2F
:10108000FBE0DF1EE11CF11CA50194010E94CB2DA9
:10109000C20ED31EE41EF51EC701B60169517C4F76
:1010A0008F4F9F4F28EE33E040E050E00E94CB2D61
:1010B000A8EEB3E00E94942DCF91FF90EF90DF90C7
:1010C000CF90BF90AF909F908F9008958F3F9105E4
:1010D00051F048F0811522E0920738F081159340D5
:1010E00030F482E0089580E0089581E0089583E07F
:1010F0000895A0E0B0E0EFE7F8E00C94172EEB01C4
:101100008A01B82FB695A0E028813981F8012083A3
:101110002A813B8121832C813D8122832E813F8145
:101120002383688179814A815B812C813D81EE81B5
:10113000FF819F2F9295990F990F907C272F2370F5
:10114000922B252F2370220F220F922B232F2370F7
:101150002295207F922BF80194830B5F1F4F2896D6
:10116000AF5FBA1788F680FF24C0888199810E94FA
:101170006608D82E8A819B810E946608E82E8C81A1
:101180009D810E946608F82E8E819F810E946608CC
:10119000F0E4DF9EA001112490E1E99E900111246A
:1011A000242B282BE4E0FE9EB0011124262BF8010D
:1011B0002083CDB7DEB7E7E00C94332E803223E0F6
:1011C000920708F1883E23E0920740F48F51934044
:1011D000E4E096958795EA95E1F70895803D27E04C
:1011E000920718F48C5D93400895883928E092079F
:1011F00068F4885C974074E0969587957A95E1F756
:101200008D509C4F089580E090E008958FEF93E01B
:1012100008958C30910540F4A4E0880F991FAA9599
:10122000E1F7885D9C4F0895843F23E0920718F40E
:1012300084529C4F0895811524E0920740F486570C
:10124000934FF4E0880F991FFA95E1F7089580E92C
:1012500098E008959C013695279525753575821B74
:10126000930B9C0123733373969587959695879579
:1012700083739373820F931F9C0154E036952795D7
:101280005A95E1F7280F391F2F703F7041E051E068
:10129000249FC001259F900D349F900D1124892F0C
:1012A00008955F98882319F00000289A02C0000072
:1012B000289800005F9A000008955F9A000083B1AB
:1012C0005F980000869581700895CF93DF93D82FA3
:1012D0005C9A5F985C98C8E08D2F80780E945109D5
:1012E000DD0FC150C9F75F98DF91CF9108958F77D7
:1012F0000E9465090895CF93DF93D82FC8E08D2F02
:1013000080780E945109DD0FC150C9F75F98DF91C5
:10131000CF910895CF93DF935F98C8E080E0D82FF6
:10132000DD0F0E945D098D0FC150C9F7DF91CF918C
:1013300008950E9477090E948A095C9A0895A1E0A5
:10134000B0E0E5EAF9E00C941C2E806869830E9405
:1013500065096981862F0E947B095C9A2196E2E0EB
:101360000C94382ECF93C0917D05C827E82FF0E06C
:10137000EC58FA4F678589E70E949F096C2F8DE32F
:101380000E949F096C2F82E40E949F09CF910895CB
:1013900086E20E9499090895CF93DF93EC016C8156
:1013A0008CE10E949F096D818DE10E949F096E81F1
:1013B0008EE10E949F096F8180E20E949F096885EB
:1013C00081E20E949F09698582E20E949F096A85E5
:1013D00083E20E949F096B8584E20E949F096C85CD
:1013E00085E20E949F096D858AE20E949F096E85B1
:1013F0008EE60E949F096F858FE60E949F0968898B
:1014000080E70E949F09698981E70E949F096A8994
:1014100082E70E949F09DF91CF910895CF92DF92DA
:10142000EF92FF92CF93DF936B017C01C11488E3AD
:10143000D8068CE9E8068CE1F80628F5C701B60164
:1014400020E836E948E950E00E94CB2DE901689791
:1014500060E879E687E69FEF0E94A72D6C0D7D1D61
:101460008E1D9F1DF2E0660F771F881F991FFA954A
:10147000D1F721E732E040E050E00E94CB2DF22E80
:10148000E32E80E421C0C701B60120E03DE241E344
:1014900051E00E94CB2DE901689760E073ED8EEC7E
:1014A0009EEF0E94A72D6C0D7D1D8E1D9F1D660F4A
:1014B000771F881F991F21E732E040E050E00E942B
:1014C000CB2DF22EE32E80E66C2F6F71680F85E72F
:1014D0000E949F096E2D86E70E949F096F2D87E766
:1014E0000E949F09DF91CF91FF90EF90DF90CF9006
:1014F0000895682F8DE60E949F0908958F929F920C
:10150000AF92BF92CF92DF92EF92FF92CF93DF9391
:10151000D82F83E00E94990980936F0584E00E9490
:10152000990980936E0560E086E00E949F0961E062
:1015300087E00E949F096FE789E00E949F0965E0AC
:101540008AE00E949F0962E18BE00E949F0965E1A9
:101550008CE00E949F096DEF8DE00E949F0960E082
:101560008EE00E949F09DD2319F08BE291E008C014
:1015700020919B0533E1239FC0011124825C9E4F83
:101580000E94CC096CE880E30E949F096FE082E32F
:101590000E949F0962E483E30E949F0980919C0559
:1015A00087FF02C064E101C06AE084E30E949F09F2
:1015B0006AE285E30E949F096DE286E30E949F092B
:1015C00064ED87E30E949F0960E088E30E949F0921
:1015D00060E089E30E949F09D11109C0C0907D0598
:1015E000D0907E05E0907F05F090800507C0C5E9AA
:1015F000CC2EC1ECDC2EED2CCEEDFC2ECAE38F2CD4
:101600009924AA24BB24682D8C2F0E949F09682D41
:1016100085E08C0F0E949F09FE2CED2CDC2CCC2445
:10162000CF5FCE3361F76FEF83E40E949F096FEFC6
:1016300084E40E949F096FEF85E40E949F096FEF89
:1016400086E40E949F09DD2311F066E002C06091EC
:1016500081058DE60E949F0960E089E70E949F094D
:10166000609182058AE70E949F0960E083E70E94FB
:101670009F0960E084E70E949F09D11109C0609131
:10168000790570917A0580917B0590917C0504C065
:1016900060EC7AEC89E896E30E940E0ADF91CF9124
:1016A000FF90EF90DF90CF90BF90AF909F908F9082
:1016B000089561E087E00E949F0964E28EE70E943E
:1016C0009F0963E088E00E949F0960E088E00E9433
:1016D0009F0965E087E00E949F0962E085E00E9423
:1016E0009F0983E00E94990980936F0584E00E941E
:1016F000990980936E05089583E00E94990980936B
:101700006F0584E00E94990980936E0561E087E08F
:101710000E949F096AE070E080E090E00E949628B5
:101720000E94590B00000895CF92DF92FF920F9311
:101730001F93CF93DF931F92CDB7DEB7082F162FDD
:101740008EE399830E949F09F02EC02E9981D92E95
:101750008C2D8F19811738F4F60161916F018FE795
:101760000E949F09F5CF64E085E00E949F0983E015
:101770000E94990980936F0584E00E9499098093E3
:101780006E050E94732860936A0570936B058093C1
:101790006C0590936D0569E087E00E949F0981E0E8
:1017A000809371050F90DF91CF911F910F91FF9062
:1017B000DF90CF9008950F931F930E94940B809118
:1017C0007105813099F40E94732800916A05109187
:1017D0006B0520916C0530916D05601B710B820BC0
:1017E000930B603A76488140910548F380917105EA
:1017F000813031F46EE971E080EE95E00E945F2A5D
:101800001F910F9108950F931F938091710582305E
:1018100021F41092710581E020C080917105813022
:10182000D9F40E94732800916A0510916B052091EC
:101830006C0530916D05601B710B820B930B613A47
:1018400076488140910540F061E087E00E949F0961
:101850001092710582E001C080E01F910F91089500
:10186000CF93DF93EC014AE050E06D2F70E080EE03
:1018700095E00E942D2B6EE280EE95E00E94312AC9
:10188000BE0184E0769567958A95E1F76F707727BA
:101890004AE050E080EE95E00E942D2B6EE280EE53
:1018A00095E00E94312ABE016F7077274AE050E030
:1018B00080EE95E00E942D2BDF91CF910895D82FD7
:1018C000C0E0CD1780F42D9A64E670E080E090E0EF
:1018D0000E9496282D9864E670E080E090E00E94D7
:1018E0009628CF5FEECF6CE271E080E090E00E943E
:1018F0009628E6CF0F931F93CF93DF93EC01062F2B
:1019000015E0115051F0CE010E942830081741F027
:10191000602FCE010E943030F4CF82E00E945F0C35
:10192000DF91CF911F910F910895A0E0B0E0EBE916
:10193000FCE00C940E2E482E562EC0E0D0E0612C18
:10194000712CE12CF12C00E010E041100CC06090F3
:10195000D20586E4689E3001112459E1E52EF12C70
:1019600008EB15E01EC091E049120FC06090D2054F
:10197000E6E46E9E30011124FBE16F0E711C49E21A
:10198000E42EF12C04E715E00CC082E0481209C0F7
:1019900028E1622E77247394EE24E394F12C01ED78
:1019A00015E043018C0E9D1E109273051092720576
:1019B0003401A62CA818B12CC30101966C01AE14F9
:1019C000BF04A8F4A00EB11E511006C0C3010E94AE
:1019D0002830F501808305C0F5016081C3010E94B4
:1019E0007A0CF50180810E9461063601E2CFC301C5
:1019F000511018C0C3010E942830B82EC6010E94A1
:101A000028302B2D30E0322F2227282B8091720591
:101A1000909173058217930779F4C0E0D0E05524C4
:101A2000539493CF3601609173050E947A0C6091B4
:101A30007205C6010E947A0CC05EDE4FC13E92E084
:101A4000D90708F482CF852DCDB7DEB7E0E10C943D
:101A50002A2E61E082E00E94950C089560E082E009
:101A60000E94950C8091D105853020F01092D1050F
:101A70000E94290D8091D1058093D205089561E0DF
:101A800080E00E94950C61E081E00E94950C089531
:101A900060E080E00E94950C882351F060E081E0D6
:101AA0000E94950C882321F080917405883349F0B9
:101AB0000E94BF060E947A0681E00E94DF060E9413
:101AC0003F0D0895882319F06AEA71E002C06EEABA
:101AD00071E080EE95E00E945F2A0895FF920F93D7
:101AE0001F93CF93DF9369EC7BE080EE95E00E943B
:101AF0000B2A4091790550917A0560917B05709190
:101B00007C052AE030E080EE95E00E94342B63EB08
:101B10007BE080EE95E00E940B2A40917D0550917C
:101B20007E0560917F057091800520E130E080EEB8
:101B300095E00E94342B6DE97BE080EE95E00E94F9
:101B40000B2A4AE050E06091810580EE95E00E940A
:101B50005C2B67E87BE080EE95E00E940B2A4AE070
:101B600050E06091820580EE95E00E945C2B61E779
:101B70007BE080EE95E00E940B2AC3E8D5E0F12CD3
:101B80008E0188818823A9F0FF2031F061EB71E09C
:101B900080EE95E00E942E2A21964AE050E0F8015E
:101BA000608180EE95E00E94252BF394F8E1FF120E
:101BB000E7CF80EE95E00E94392A6BE57BE080EE6E
:101BC00095E00E940B2A4AE050E060919B0580EE70
:101BD00095E00E945C2B66E47BE080EE95E00E943D
:101BE0000B2AE0919C05E770F0E0EE0FFF1FEE5727
:101BF000FC4F6081718180EE95E00E945F2A61E375
:101C00007BE080EE95E00E940B2A80919C05887114
:101C1000883069F028F4811113C068E27BE00CC0C1
:101C2000803141F0883161F46CE07BE005C06CE10B
:101C30007BE002C066E17BE080EE95E00E944D2AE9
:101C400068EF7AE080EE95E00E940B2A40917505DE
:101C50005091760560917705709178052AE030E023
:101C600080EE95E00E94342B6FED7AE080EE95E0F7
:101C70000E940B2A8091BD0580710E94620D66EC66
:101C80007AE080EE95E00E940B2A8091BD05807479
:101C90000E94620D6DEA7AE080EE95E00E940B2AC8
:101CA0008091BD0580720E94620D60E97AE080EE4D
:101CB00095E00E940B2A84E795E00E94F407AB01AF
:101CC000BC012AE030E080EE95E00E94162B6BE824
:101CD0007AE080EE95E00E940B2A84E795E00E946E
:101CE000F4079B01AC0160E472E48FE090E00E9495
:101CF000CB2DBA01A9012AE030E080EE95E00E94E8
:101D0000162B68E87AE080EE95E00E944D2ACDB768
:101D1000DEB7E5E00C94352E8F929F92AF92BF9282
:101D2000CF92DF92EF92FF92811107C06FE77AE0C6
:101D300080EE95E00E944D2A2FC090E00E9474072B
:101D400024E630E040E050E00E94CB2DCA01B9010A
:101D50002AE030E040E050E00E94CB2D49015A01DA
:101D60006B017C012AE030E0B501A40180EE95E032
:101D70000E94162B6EE280EE95E00E94312A2AE046
:101D800030E0B701A60180EE95E00E94162B63E7D4
:101D900080EE95E00E94712AFF90EF90DF90CF9047
:101DA000BF90AF909F908F9008951F93CF93DF9334
:101DB00065E77AE080EE95E00E940B2A80919D0510
:101DC000813041F46CE57AE080EE95E00E944D2A86
:101DD00010E050C0823019F465E47AE0F5CF843029
:101DE00019F461E37AE0F0CF853091F766E27AE0AA
:101DF000EBCFC12FD0E0C930D1050CF441C068E36E
:101E0000610F80EE95E00E94312A6EE17AE080EE6B
:101E100095E00E940B2ABE016F5F7F4F4AE050E0C1
:101E200080EE95E00E94F52A63E17AE080EE95E08D
:101E30000E940B2AC356DA4FE981E03218F566E0BA
:101E40007AE080EE95E00E940B2A8981803130F0A3
:101E50006DE673E080EE95E00E942E2A69816F7036
:101E600070E06F5F7F4F4AE050E080EE95E00E94A7
:101E7000FE2A1F5F80914605181708F4BACF0FC0DD
:101E800061E3BECFEF70F0E0EE0FFF1FEE56FC4FA8
:101E90006081718180EE95E00E945F2AEACF6BEE4F
:101EA00079E080EE95E00E940B2A8091B5050E94B2
:101EB0008C0E60ED79E080EE95E00E940B2A809117
:101EC000B6050E948C0E65EB79E080EE95E00E94ED
:101ED0000B2A8091B7050E948C0E6AE979E080EEAA
:101EE00095E00E940B2A4091AD055091AE0560919E
:101EF000AF057091B005411551056105710539F1C6
:101F00002AE030E080EE95E00E94342B67E679E02D
:101F100080EE95E00E940B2A8091B1050E949907FE
:101F2000AB01BC012AE030E080EE95E00E94342B4A
:101F300063E479E080EE95E00E940B2A4AE050E0ED
:101F40006091B20580EE95E00E945C2B06C06AE3CA
:101F500079E080EE95E00E944D2A6DE179E080EE17
:101F600095E00E940B2A6091B3057091B4054AE098
:101F700050E080EE95E00E94462B60E079E080EE34
:101F800095E00E940B2A6091AC05603450F470E03B
:101F90006F5F7F4F4AE050E080EE95E00E94FE2A9E
:101FA00006C067EF78E080EE95E00E944D2A6AED6A
:101FB00078E080EE95E00E940B2A8091AB0580FFCF
:101FC00003C063EB71E002C067EB71E080EE95E067
:101FD0000E945F2A6DEB78E080EE95E00E940B2A6C
:101FE0008091AB0582700E94620D6EE978E080EE10
:101FF00095E00E940B2A8091AB0584700E94620DCF
:102000006FE778E080EE95E00E940B2A8091AB05A7
:1020100088700E94620DDF91CF911F9108950F93F8
:102020001F93CF93DF93209143052F3FA9F56FEFC7
:1020300075E080EE95E00E940B2A82E893E00E9412
:10204000300C6EED75E080EE95E00E940B2A8091D9
:102050004405909145050E94300C6BEA75E080EED6
:1020600095E00E944D2A68E875E080EE95E00E94B8
:102070004D2A60E775E080EE95E00E944D2A6BE402
:1020800075E080EE95E00E944D2A80EE95E00E947A
:10209000392A0E94D50E68C012160CF065C033278D
:1020A00027FD30958091460590E0821793070CF448
:1020B0005BC066E375E080EE95E00E940B2A6091BC
:1020C0004305772767FD70954AE050E080EE95E084
:1020D0000E94FE2A6BE075E080EE95E00E940B2ADC
:1020E00010E008E2809147051817D0F5C12FD0E025
:1020F000CC0FDD1FC85BDA4F288130E080914305AB
:10210000992787FD909501972817390739F56BEBCB
:1021100071E080EE95E00E942E2A4AE050E0602FA8
:1021200080EE95E00E94252B6FEB71E080EE95E04C
:102130000E942E2AE981EF70F0E0EE0FFF1FEE56AD
:10214000FC4F6081718180EE95E00E942E2A63EC45
:1021500071E080EE95E00E942E2A0F5F1F5FC2CFD4
:1021600080EE95E00E94392ADF91CF911F910F9167
:102170000895FF920F931F93CF93DF93C3E8D5E0A9
:10218000F12C8E0188818823D1F165EC71E080EE1D
:1021900095E00E942E2A4AE050E06F2D80EE95E0F7
:1021A0000E94252B62ED71E080EE95E00E942E2AC0
:1021B0002196F801208130E0A0E1B7E20E94852D50
:1021C0009B01AC01A0918205B0E00E94942DAB016F
:1021D000BC018091790590917A05A0917B05B09121
:1021E0007C05480F591F6A1F7B1F2AE030E080EEF4
:1021F00095E00E94342BF394F8E1FF12C2CFCDB7E3
:10220000DEB7E5E00C94352E1092DD0485E6EEEDA8
:10221000F4E0DF011D928A95E9F70895CF93C82F66
:102220008F3719F0883009F045C0E091DD04EE23C6
:10223000D9F1E150E093DD04F0E0E252FB4F10826F
:102240006DE070E080EE95E00E945906C0E080915C
:10225000DD04C81760F4EC2FF0E0E252FB4F608120
:1022600070E080EE95E00E945906CF5FF0CF60E20B
:1022700070E080EE95E00E9459066DE070E080EE1F
:1022800095E00E945906C0E08091DD04C81778F5FA
:10229000EC2FF0E0E252FB4F608170E080EE95E0C1
:1022A0000E945906CF5FF0CF67E080EE95E00E9474
:1022B000312A1DC08B3119F40E9404111AC08D30CF
:1022C000C1F08A30B1F08091DD04843668F76C2F5C
:1022D00070E080EE95E00E945906E091DD0481E017
:1022E0008E0F8093DD04F0E0E252FB4FC08380E06C
:1022F00001C081E0CF910895CF93C82F0E94732829
:102300006093C6047093C7048093C8049093C90473
:10231000C093DB04CC2329F040E051EE60E070E094
:1023200004C040E855E260E070E080EE95E00E9475
:10233000BB2CCF9108959091CA04492F4F7050E063
:10234000BA016F5F7F4F292F30E0E4E03595279584
:10235000EA95E1F76217730759F0FA01E553FB4F6D
:10236000808381E0890F8F70907F892B8093CA04CE
:1023700008956EE770E080EE95E00E94590608959A
:10238000A3E1B1E0E6ECF1E10C940F2EE3E8F5E017
:10239000712C8191882321F0739428E17212F9CF76
:1023A00066ED71E080EE95E00E945F2A4AE050E021
:1023B000672D80EE95E00E945C2B80E00E947E0AF3
:1023C0000E94590B8E010E5F1F4FC12CD12C76013C
:1023D000C39466246A945C2C0E9467284B015C01BC
:1023E0002091820530E0A0E1B7E20E94852D9B019B
:1023F000AC01C701B6010E94A72D2091790530914B
:102400007A0540917B0550917C05620F731F841FF4
:10241000951F2091B9053091BA054091BB055091A7
:10242000BC05261737074807590718F4F8016082DA
:1024300025C08C2D0E94B20961E070E080E090E040
:102440000E949628F80110820E946728681979096D
:102450008A099B09643F71408105910540F40E94FF
:10246000C809F8019081981778F78083EDCF50FE66
:1024700003C02C982D9A02C02C9A2D982FEFC21AC7
:10248000D20AE20AF20A0F5F1F4F8FEFC816D1047B
:10249000E104F10409F09FCFCE019395FC01D82E01
:1024A0007FEF68EC2E2F281B271510F051E056C047
:1024B000DE01129651E02FEF41E03D91321710F00E
:1024C000322F01C0452F5F5F5F3F11F0232FF5CF03
:1024D0004193242F30E0A1E0B0E0AC0FBD1FA20F6C
:1024E000B31F5C93413079F0DE01A20FB31F5C9300
:1024F000423049F0AFEFBFEFAC0FBD1FA20FB31FCB
:102500006C934E3F78F6A2E0B0E0AC0FBD1FA20F77
:10251000B31F7C934D3F30F6A3E0B0E0AC0FBD1F7E
:10252000A20FB31F6C93BECF452F242F30E0FC01C8
:10253000E20FF31F6081AFEFB0E0AC0FBD1FA20F41
:10254000B31F2C91621748F44150DC01A40FB11D58
:102550002C9120836C934111E8CF5F5F571520F3D6
:10256000372D369520E0231770F4DC01A20FB11D42
:102570004C91522F530FFC01E50FF11D50815C93DC
:1025800040832E5FF0CFF3E8EF2EF5E0FF2E8C01B5
:10259000802F8D19871598F4F801C1908F014AE0BA
:1025A00050E06C2D80EE95E00E94252B6CE280EED1
:1025B00095E00E94312AF701C1927F01E9CF80EEB8
:1025C00095E00E94392A81E0CD5EDE4FEFE00C9469
:1025D0002B2E1F920F920FB60F9211240F931F9361
:1025E0002F933F934F935F936F937F938F939F931B
:1025F000AF93BF93EF93FF934091BD055091BE05FC
:102600006091BF057091C00589B18A019B0100747A
:1026100011272227332783FB882780F990E0A0E049
:10262000B0E0081719072A073B0709F468C0809132
:102630008400909185001092850010928400209172
:10264000A70421115CC045FD02C096958795853C85
:1026500029E09207C0F180910A0190E0A0E0B0E08B
:102660000CE176956795579547950A95D1F74115F1
:1026700051056105710521F441E050E060E070E032
:10268000481759076A077B07D8F480910A018F3FE2
:10269000B9F040E080910A01481780F4842F90E05F
:1026A000880F991FFC01E957FB4F20813181FC0104
:1026B000E55FFE4F318320834F5FECCF1092A8047B
:1026C00010920A011CC08D3B22E09207A8F02091D5
:1026D0000A01203188F410910A0121E0210F209392
:1026E0000A010E94DE08E12FF0E0EE0FFF1FE9571C
:1026F000FB4F9183808303C08FEF80930A01FF918A
:10270000EF91BF91AF919F918F917F916F915F9169
:102710004F913F912F911F910F910F900FBE0F90EE
:102720001F90189583E0809380008AE18093810058
:102730008FEF9FEF909389008093880010926F0035
:1027400088E080936D00E8E6F0E08081846080831B
:1027500008950E942E0D8091D205843011F41092BC
:10276000D20508956F3018F086958058089589E055
:10277000689F802D11240895A0E0B0E0E2ECF3E121
:102780000C94162EC82F0E947328009138041091C3
:10279000390420913A0430913B046B017C01C01A4A
:1027A000D10AE20AF30A9701860149E8C41643E117
:1027B000D406E104F10410F010923C046093380454
:1027C0007093390480933A0490933B042091A704BA
:1027D0008FEF820F8230D8F5E0913C04EE2309F4AC
:1027E0004EC1E13011F482E0B8C1E03108F034C1EB
:1027F00081E08E0F80933C04F0E0E957FB4FC083EB
:10280000803109F0ACC1E9E8F4E0213029F4A1817C
:10281000A695A695808108C080819181A92FA69553
:10282000A695A69596958795A03148F4B0E090E0DE
:10283000AA0FBB1FA55FBE4F11969C938E9310925B
:10284000A804329684E0E739F807F9F688C1233006
:1028500009F005C1E0913C04E11104C0CF3009F05A
:102860007EC10DC1E83148F481E08E0F80933C04B5
:10287000F0E0EA57FB4FC08372C1E83109F0ECC0C9
:10288000C111EAC040E050E0ABE0CA01B3E0880FFC
:10289000991FBA95E1F7A49F9001A59F300D1124CF
:1028A000F901E957FB4F6081E1817E2F77707595C3
:1028B0006795FC01EE0FFF1FE55FFE4F718360839C
:1028C000F901E857FB4FB081B695B695B695E18111
:1028D000FE2FF295FF0FF07E6F2F6B2BE695E6959E
:1028E000E6957E2F777075956795FC01EE0FFF1FBB
:1028F000E35FFE4F71836083F901E757FB4FB081BF
:10290000B295B695B695B370C181DC2FDD0FDD0FA2
:102910006D2F6B2BC295C695C695C370E281E17091
:10292000EE0FEE0F7E2F7C2B75956795FC01EE0F59
:10293000FF1FE15FFE4F71836083F901E557FB4F95
:10294000B081B695E181FE2FF795FF27F7956F2FA0
:102950006B2BE6957E2F777075956795FC01EE0FD2
:10296000FF1FEF5EFE4F71836083F901E457FB4F59
:10297000B081B295BF70E181FE2FF295F07F6F2F8D
:102980006B2BE295EF707E2F777075956795FC0144
:10299000EE0FFF1FED5EFE4F71836083F901E35779
:1029A000FB4FB081BB1FBB27BB1FC181DC2FDD0FDD
:1029B0006D2F6B2BCC1FCC27CC1FE281E370EE0F69
:1029C0007E2F7C2B75956795FC01EE0FFF1FEB5E4C
:1029D000FE4F71836083F901E157FB4FB081B695DB
:1029E000B695E181FE2FF295FF0FFF0FF07C6F2F60
:1029F0006B2BE695E6957E2F777075956795FC01B4
:102A0000EE0FFF1FE95EFE4F71836083F901E0570F
:102A1000FB4F20812295269527703181E32FEE0F01
:102A2000EE0FEE0F6E2F622B732F729576957770E7
:102A300075956795FC01EE0FFF1FE75EFE4F7183F2
:102A400060834F5F5F4F4230510509F01ECF809188
:102A50009D0483FF1092A80410923C0480C024308F
:102A600009F07DC060913C0461110BC0C83AB1F41B
:102A7000109273051092720588EA0E94610681E047
:102A80006CC0613019F4C093370404C0623031F473
:102A9000C09336048C2F0E9461065AC0E091360420
:102AA0002E2F30E0220F331F462F50E0C90102962F
:102AB000841795073CF0633268F7FA01EC57FB4F37
:102AC000C083E8CF2D5F3F4F8C2F90E0609172055F
:102AD000709173054217530749F4982F882786276A
:102AE0009727909373058093720532C06817790712
:102AF00069F580913704813049F5E13118F080E1C2
:102B000080933604F0903604C8E8D4E000E010E08A
:102B10000F15D0F4FE013197808190E0982F88271F
:102B20002881822B43E0969587954A95E1F70E948C
:102B3000DE08F801EE0FFF1FE55FFE4F91838083F3
:102B40000F5F1F4F2296E4CF1092A80410923C040E
:102B500080913C04882319F08F5F80933C04CDB7AB
:102B6000DEB7E8E00C94322EE82FF0E0E854FA4F9C
:102B7000E185E03150F4F894F0E0EE0FFF1FE55FDF
:102B8000FE4F8081918178940895E03121F0E13108
:102B900031F483E101C082E10E94B529089580E00B
:102BA00092E00895A2E2B0E0E8EDF5E10C940C2E7D
:102BB0009E012F5F3F4F80E1D9011D928A95E9F771
:102BC00064E072E080EE95E029A33AA30E945F2AB8
:102BD0000E947C0B1D8A1E8A1F8A188E312C212C84
:102BE00000E0812C912C540170EC472E7DE9572E8A
:102BF00078E5672E75E3772EE0E5CE2EE3ECDE2E4A
:102C0000E12CF12C84EF91E0A0E0B0E08D8F9E8F5D
:102C1000AF8FB8A380EC97EFAAEBB7E3898F9A8FB9
:102C2000AB8FBC8F80EC9DE9A8E5B5E3898B9A8BCF
:102C3000AB8BBC8B80EE95E00E94732B892B09F443
:102C4000E1C080EE95E00E94A02B9C0133272C323E
:102C5000310509F442C0ACF42332310509F0ABC0B0
:102C600019821A821B821C821D821E821F82188674
:102C700019861A861B861C861D861E861F86188A44
:102C800060C02434310529F02335310509F4B2C080
:102C900092C064E480EE95E00E94312A2AE030E0A0
:102CA00040EC5DE968E575E380EE95E00E94BF2A9F
:102CB0006CE280EE95E00E94312A2AE030E040ECA0
:102CC00057EF6AEB77E380EE95E00E94BF2A6CE253
:102CD00080EE95E00E94712AADCF0F5F043009F0BD
:102CE000A9CF29813A814B815C81A8EEB3E00E9493
:102CF000942D698B7A8B8B8B9C8B2D813E814F81A0
:102D000058850E94942D698F7A8F8B8F9C8F29858F
:102D10003A854B855C852D8F3E8F4F8F58A32D852F
:102D20003E854F8558890E94942D6B017C0160324D
:102D30003EE473078105910530F462E38CE10E9463
:102D40009F0900E077CF603345E77407810591055F
:102D500010F462E2F3CF60345CE9750781059105F8
:102D600010F466E2EBCF80E5C81683ECD806E104E8
:102D7000F10410F462E1E2CF90E6C9169AEED906AA
:102D8000E104F10410F465E1D9CFA0E7CA16A1E18E
:102D9000DA06A1E0EA06F10410F461E0CFCFB0EA70
:102DA000CB16B6E8DB06B1E0EB06F10410F463E005
:102DB000C5CF65E0C3CF10ED180F1A3008F03ACF39
:102DC000E1E0F0E0EC0FFD1F24E0029FE00DF11DBB
:102DD00011242081318142815381AAE0B0E00E9418
:102DE000942D610F711D811D911D608371838283FC
:102DF000938320CF49885A886B887C88812C912CBA
:102E0000540118CF81149104A104B10489F4C301C1
:102E1000B2010E940E0A61E070E080E090E00E9442
:102E200096281D8A1E8A1F8A188E312C22242A94E5
:102E30008D8D9E8DAF8DB8A188169906AA06BB060A
:102E4000D0F40E94C8092D893E894F89588D280FDA
:102E5000311D411D511D2D8B3E8B4F8B588F3816C8
:102E600008F4382E821508F4282E3FEF831A930AAF
:102E7000A30AB30A56C0C301B20128EE33E040E012
:102E800050E00E94CB2DBA01A9012AE030E080EE8B
:102E900095E00E94162B6CE280EE95E00E94312AAC
:102EA0004AE050E0632D80EE95E00E94252B6CE215
:102EB00080EE95E00E94312A6D897E898F89988DF8
:102EC000A50194010E94CB2DBA01A9012AE030E0AE
:102ED00080EE95E00E94162B6CE280EE95E00E9459
:102EE000312A4AE050E0622D80EE95E00E94252BC9
:102EF0006CE280EE95E00E94712A4C0C5D1C6E1C09
:102F00007F1C898D9A8DAB8DBC8D84159505A6058A
:102F1000B70520F449885A886B887C88812C912CCD
:102F2000540129893A894B895C89283E33404105FF
:102F3000510509F07FCEA296E2E10C94282EACE177
:102F4000B0E0E5EAF7E10C94162E0E9473286B01BD
:102F50007C0181E00E947E0A14E703E0198361E0AE
:102F6000CE0101960E94DB0B009371050E94590B64
:102F70006AEF70E080E090E00E94962880917105F1
:102F8000833089F480EE95E00E94732B892B59F4ED
:102F90000E9473286C197D098E099F096038734C53
:102FA000894C9140D8F280917105833009F44FC06B
:102FB0008FE70E9477090E948A098983843511F07E
:102FC00083E05CC00E948A09109244058093450505
:102FD0000E948A092091440530914505280F311D32
:102FE00030934505209344050E948A098093460545
:102FF0000E948A0980934705813110F7F12C0F2D2B
:1030000010E08091470590E0880F991F0817190775
:1030100040F40E948A09F801E85BFA4F8083F39438
:10302000EECF80E7898361E0CE0101960E94DB0B41
:1030300083E0809371050E94590B62E370E080E0A9
:1030400090E00E94962880917105833011F482E00F
:1030500015C08FE70E9477090E948A09898380350D
:1030600009F0AECF0DE915E00E948A09F8018193BD
:103070008F01F5E0083B1F07B9F781E06C96E8E0A7
:103080000C94322E80914305992787FD9095A92FA6
:10309000B92FFC013196EB30F10508F066C0EC5C0D
:1030A000FF4F0C94432E62E778E080EE95E00E949B
:1030B0004D2A82E893E00E94300C6AE578E080EEC9
:1030C00095E00E944D2A65E378E080EE95E00E944D
:1030D0004D2A6BE078E080EE95E00E944D2A6AEE82
:1030E00077E080EE95E00E944D2A6DEB77E080EE70
:1030F00095E00E944D2A67E977E080EE95E00E9416
:103100004D2A63E777E080EE95E00E944D2A6CE45B
:1031100077E080EE95E00E944D2A80EE95E00E94D7
:10312000392A0E946E0D21C06FE277E01AC06AE072
:1031300077E017C065EF76E014C066ED76E011C069
:1031400062E976E00EC06DE776E00BC068E676E0F7
:1031500080EE95E00E944D2A62E276E002C06CE0CB
:1031600076E080EE95E00E944D2A6AE070E080E013
:1031700090E00E94962880EE95E00E94732B892BA8
:1031800029F080EE95E00E94A02BF5CF0895ACE1E8
:10319000B0E0EDECF8E10C94162E909143059F3FC2
:1031A00009F023C1482F50E0FA013A97EF36F105B4
:1031B00008F00FC1E15CFF4F0C94432E61E172E017
:1031C000A0C06DE172E080EE95E00E945F2A85E785
:1031D00089838BE1EDE9F5E0DE01129601900D9215
:1031E0008A95E1F76CE1CE0101960E94DB0B0E940B
:1031F000590B83E08093710568EC70E080E090E00B
:103200000E94962880917105843009F0E2C08FE712
:103210000E9477090E948A098983853509F0D9C0FF
:103220006DEE74E080EE95E00E944D2A6FEC74E044
:1032300080EE95E00E944D2A61EB74E096C065E354
:1032400072E080EE95E00E945F2A89E6898361E062
:10325000CE0101960E94DB0B0E94590B83E0809304
:10326000710568EC70E080E090E00E949628809103
:103270007105843009F0ADC08FE70E9477090E9484
:103280008A0989838E010E5F1F4F7E014DE1E40E96
:10329000F11C0E948A09F80181938F01EE15FF0548
:1032A000C1F78BE1FE013296ADE9B5E001900D92D8
:1032B0008A95E1F78981893409F08BC063E974E06C
:1032C00080EE95E00E944D2A65E774E080EE95E07F
:1032D0000E944D2A67E574E048C06FE472E080EE1A
:1032E00095E00E945F2A8EEF8093430572C0805262
:1032F0008750805390914605981708F066C06EE598
:1033000072E080EE95E00E945F2A63C084E18093C2
:10331000430560E274E029C085E18093430569EECE
:1033200073E023C086E18093430562EB73E01DC028
:1033300087E18093430568E673E017C088E18093D6
:10334000430567E573E011C089E18093430563E4B9
:1033500073E00BC08AE1809343056EE273E005C021
:103360008BE18093430566E073E080EE95E00E9478
:103370004D2A2FC06CEE72E080EE95E00E944D2A3F
:103380008091AB0591E01DC066ED72E080EE95E0A6
:103390000E944D2A8091AB0592E013C061EC72E06F
:1033A00080EE95E00E944D2A8091AB0594E009C023
:1033B00066EA72E080EE95E00E944D2A8091AB05AE
:1033C00098E089278093AB058FEF809343050E9497
:1033D0000F1080EE95E00E94732B892B09F45BC1DE
:1033E00080EE95E00E94A02BF4CF0E940E1188235E
:1033F00009F451C18091DD04811104C08FEF8093E5
:10340000430541C140E050E060E070E08EED94E0A3
:103410000E94BA2E40914305042F112707FD1095F5
:10342000212F312FF8013197EB31F10508F01BC145
:10343000E255FF4F0C94432E552747FD50952091A0
:10344000460530E0241735070CF40DC18B019C01B3
:1034500001501109210931090032110521053105F9
:1034600058F0C0904705E9E4F5E0F12CD12CA8E232
:10347000EA2E415051090FC0FA01E356FA4F61504C
:103480006083D9C0DF0111972C9130E024173507F4
:1034900029F0F3943296FC10F5CFCBC00E2D10E03E
:1034A00020E030E0061717072807390741F420818C
:1034B000DA01A356BA4F11962C93DD24D394E394EA
:1034C000E8CF6F3F71058105910511F008F0CBC081
:1034D0006093B505B0C06F3F71058105910511F08E
:1034E00008F0C1C06093B605A6C06F3F71058105A5
:1034F000910511F008F0B7C06093B7059CC020910A
:10350000DE0420622037E9F440E050E060E070E043
:103510008FED94E00E94BA2E9B01AC01DC01CB013F
:103520000197A109B1090897A105B10508F0AEC03E
:10353000A4EDB0E30E94942D6A5E7C4A8A46954EC3
:1035400024C02636E9F440E050E060E070E08FED02
:1035500094E00E94BA2E9B01AC01DC01CB010197E3
:10356000A109B1090797A105B10508F08FC0A8EA24
:10357000B1E60E94942D645E7C438E46944E05C055
:10358000611571058105910579F08B019C01005C45
:103590001D49284535430130FAE51F07F2E62F079C
:1035A000F2E03F0708F05FC06093AD057093AE0591
:1035B0008093AF059093B0053EC06F3F71058105C4
:1035C000910511F008F04FC06093B10534C08B0134
:1035D0009C0101501109210931090F3F11052105F5
:1035E000310508F040C06093B20525C08B019C01F5
:1035F000045C1940210931090D344DE114072105FE
:10360000310528F47093B4056093B30514C06115B7
:1036100071058105910521F48FEF8093AC050BC0F6
:103620006134710581059105F0F461506093AC053A
:1036300002C0DD20C1F08091DC0481111AC08091AC
:103640007D0590917E05A0917F05B0918005019642
:10365000A11DB11D80937D0590937E05A0937F05EC
:10366000B093800506C060E772E080EE95E00E94AE
:103670005F2A0E9404118FEF809343056AE080EE79
:1036800095E00E94712A0E940F1005C061E070E071
:1036900080E090E07ACF6C96E8E00C94322E6AE5F8
:1036A00072E080EE95E00E944D2A62E472E080EEC6
:1036B00095E00E944D2A80EE95E00E94732B892BA5
:1036C00031F080EE95E00E94A02B0E94C7180E9466
:1036D0009F17823029F0833051F46DE072E002C010
:1036E00064E272E080EE95E00E944D2A08958FEF2B
:1036F000809343051092DC040E940F1080914305D3
:103700008E3F69F080EE95E00E94732B892BB1F318
:1037100080EE95E00E94A02B0E94C718EFCF08957D
:103720000F931F93109143051F3F09F0D2C08934B6
:1037300009F457C000F5883309F469C058F48033A0
:1037400009F477C008F061C08B3109F440C08132C0
:10375000B1F1B9C0813409F487C030F4893309F478
:1037600066C0803461F1AFC0823409F48EC0863403
:1037700009F448C0A8C0823609F487C078F48835B7
:1037800031F128F48235C1F18335E1F09CC08A35EE
:1037900009F494C0813609F467C095C0823761F19D
:1037A00028F4863679F18936E1F08DC0883779F0D2
:1037B0008A3709F483C0833709F085C003C061E10B
:1037C00072E015C00E943F0D6EE872E004C00E94D6
:1037D000480D68EA72E080EE95E00E945F2A8EEF65
:1037E00070C00E947A060E94BF0667EC72E080EE0D
:1037F00095E00E945F2A67C081E00E94DF0660EECC
:1038000072E0F5CF0E94B9105EC080535AC06AEFD3
:1038100071E080EE95E00E944D2A90919C0588E031
:10382000890F8871977E892B80939C051AC089E047
:1038300048C067EE71E080EE95E00E944D2A8091CD
:10384000BD059091BE05A091BF05B091C00520E1D6
:1038500082278093BD059093BE05A093BF05B093CA
:10386000C005109343052FC061ED71E080EE95E037
:103870000E944D2A8091BD059091BE05A091BF0583
:10388000B091C00540E4842710C060EC71E080EE88
:1038900095E00E944D2A8091BD059091BE05A091B2
:1038A000BF05B091C00520E282278093BD059093AB
:1038B000BE05A093BF05B093C00502C00E944F1B78
:1038C0008FEF80934305809143058E3F09F0D4C06C
:1038D000DDC00E940E11882309F4D8C08091DD0458
:1038E000811104C08FEF80934305C6C040E050E0D3
:1038F00060E070E08EED94E00E94BA2E00914305E6
:10390000112707FD1095212F312FF8013197E9304C
:10391000F10508F0B4C0E753FF4F0C94432E8B0120
:103920009C01015C1D49284535430F3F194522463E
:10393000324008F0A4C06093790570937A058093B3
:103940007B0590937C0577C060937D0570937E0521
:1039500080937F059093800581E08093DC046BC0A9
:10396000683071058105910508F089C06093810573
:1039700062C08B019C0101501109210931090A30F3
:1039800011052105310508F07AC06093820553C006
:1039900061EB71E08EED94E00E94F42F10E000974F
:1039A00099F00E94CE2F009779F0183130F4E12F72
:1039B000F0E0EC58FA4F87871F5F61EB71E080E021
:1039C00090E00E94F42FEBCF1831A8F5E12FF0E042
:1039D000EC58FA4F17861F5FF7CF653071058105E8
:1039E000910508F04CC060939B0525C08B019C019C
:1039F0000150110921093109063011052105310550
:103A0000F0F520919C05287F262B20939C0513C060
:103A10008B019C0101501109210931090115124C3A
:103A20002140310560F560937505709376058093AC
:103A30007705909378058091DC04811113C0809103
:103A40007D0590917E05A0917F05B091800501963E
:103A5000A11DB11D80937D0590937E05A0937F05E8
:103A6000B09380050E9404118FEF809343056AE0B4
:103A700080EE95E00E94712A0E94421807C060E71C
:103A800072E080EE95E00E945F2AECCF1F910F91CB
:103A900008958FEF809343051092DC040E94421832
:103AA000809143058E3F69F080EE95E00E94732B74
:103AB000892BB1F380EE95E00E94A02B0E94901B11
:103AC000EFCF6AE070E080E090E00E94962880EE00
:103AD00095E00E94732B892B29F080EE95E00E94DF
:103AE000A02BF5CF0895CF93C82F682F80EE95E0D7
:103AF0000E94CD2B909168059C2790936805CF91EB
:103B00000895A1E0B0E0E7E8FDE10C941C2E998354
:103B10000E94731D9981892F0E94731D2196E2E0F6
:103B20000C94382E1F93CF93DF93182FEB01109234
:103B3000680565EB70E080EE95E00E94590662E64C
:103B400070E080EE95E00E945906812F0E94731D5F
:103B5000CE010E94811DDF91CF911F910895609148
:103B6000680580EE95E00E94CD2B0895A1E2B0E0BB
:103B7000ECEBFDE10C94182E7B018A018C3009F4EA
:103B800053C108F040C0863009F4BCC018F583303A
:103B900009F491C070F4813009F472C0823009F0E8
:103BA00048C26BE170E082E00E94921D0DE915E0D1
:103BB00078C0843009F487C0853009F03AC260913A
:103BC000470570E0660F771F85E00E94921D08E4AC
:103BD00015E086C0893009F4A7C070F4873009F475
:103BE0009BC0883009F025C261E070E088E00E9447
:103BF000921D8091D20523C28A3009F4CAC08B304D
:103C000009F4F2C016C28A3609F475C1D8F48736B1
:103C100009F43AC138F4853609F40EC1863609F440
:103C20001FC107C2883609F437C1893609F001C2BD
:103C300061E070E089E60E94921D0E947A060E946F
:103C4000BF06F5C18D3609F4D4C138F48B3609F4BA
:103C500091C18C3609F49AC1ECC18E3609F4DCC1ED
:103C6000873C09F0E6C161E070E087EC0E94921D9C
:103C700081E00E94731D0E94AF1D10926905E3C18F
:103C800069E270E081E00E94921D04E715E0F8010E
:103C900081918F010E94731DF5E00D391F07B9F75F
:103CA000D0C1F80181918F010E94731DF5E0083B9E
:103CB0001F07B9F7C6C161E070E083E00E94921D62
:103CC0000E949F17BCC161E070E084E00E94921DD9
:103CD00081E00E94731D0E94AF1D0E94D215B3C1E6
:103CE0008091470590E0880F991F9801285435402E
:103CF0002817390708F0A5C1F80181918F010E94AA
:103D0000731DEECF62E070E086E00E94921D82E8B3
:103D100093E00E94811D95C161E070E087E00E9400
:103D2000921D809146058BC186E6898361E0CE01B4
:103D300001960E94DB0B0E94590B83E08093710572
:103D400068EC70E080E090E00E9496288091710518
:103D50008430D9F48FE70E9477090E948A09898309
:103D6000863469F460E270E089E00E94921D10E2FE
:103D70000E948A090E94731D1150D1F762C161E04F
:103D800070E089E00E94921D52C161E070E089E01C
:103D900053C169E170E08AE00E94921D82E0809345
:103DA000B805209170058091BD059091BE05A09148
:103DB000BF05B091C005222311F0806801C08F7744
:103DC0008093BD059093BE05A093BF05B093C00539
:103DD00008EB15E0F80181918F010E94731DF5E059
:103DE000013D1F07B9F72DC161E270E08BE00E9431
:103DF000921D8091A8048F3F39F08091A80491E032
:103E0000980F9093A80402C08091A8040E94731D8B
:103E100010E0812F0E94B4150E9409090E94811DA3
:103E20001F5F1031B1F70DC161E070E08CE00E94BE
:103E3000921D8091D10503C161E070E085E60E948A
:103E4000921D89E2E816F10409F0F8C0D801E4E710
:103E5000F5E08D91819385E0ED39F807D1F7E7C062
:103E600061E070E086E60E94921DEBE1EE16F1043F
:103E700009F0E4C0D801EDE9F5E08D91819385E08A
:103E8000E83BF807D1F7D3C061E070E087E60E9415
:103E9000921D0E943F0DCBC061E070E088E60E9459
:103EA000921D85E789838BE1EDE9F5E0DE0112964D
:103EB00001900D928A95E1F76CE1CE0101960E9486
:103EC000DB0B0E94590B83E08093710560E273E085
:103ED00080E090E00E94962880917105843009F07E
:103EE000ADC08FE70E9477090E948A0989838535D2
:103EF00009F0A4C09CC061E070E08AE60E94921DB7
:103F000089E6898361E0CE0101960E94DB0B0E9465
:103F1000590B83E08093710560E273E080E090E0EC
:103F20000E94962880917105843009F087C08FE740
:103F30000E9477090E948A0989838E010E5F1F4FB4
:103F40007E01EDE1EE0EF11C0E948A09F8018193D9
:103F50008F01EE15FF05C1F78BE1FE013296ADE949
:103F6000B5E001900D928A95E1F78981893409F0D5
:103F700065C05DC061E070E08BE60E94921DF801B3
:103F800080818093D2050E94480D51C061E070E0AD
:103F90008CE60E94921DF0E2EF16F10461F487E6D0
:103FA000898380E2F801DE01129601900D928A95D4
:103FB000E1F761E203C087E4898361E0CE01019605
:103FC0000E94DB0B0E94590B83E0809371056CE427
:103FD00074E080E090E00E94962880917105843022
:103FE00069F58FE70E9477090E948A09873431F5C5
:103FF0001EC061E070E08DE60E94921D89E1E81626
:10400000F104E1F4D801E8EBF5E08D91819385E0CE
:10401000E13DF807D1F70BC061E070E08EE60E9449
:10402000921DF80180818093D1050E94290D81E0C5
:1040300006C061E070E08AEC0E94921D80E00E9460
:10404000731D0E94AF1DA196E6E00C94342EA0E0F3
:10405000B0E0EDE2F0E20C94162ECAECD3E014E6E8
:1040600006E035E0F32E44E0E42E53E0D52E62E086
:10407000C62E80EE95E00E94732B892B09F49BC01D
:1040800080EE95E00E94A02B282F8093350440916C
:10409000340450E04730510560F7FA01EE52FF4F0B
:1040A0000C94432E853B29F781E080933404E1CFC3
:1040B000823609F07DC0C0923404DBCF8093330494
:1040C00080933204D0923404D4CF9C0133273093B0
:1040D0003104209330049091320498279093320455
:1040E000E0923404C6CF382F2227409130045091FB
:1040F0003104242B352B30933104209330049091DC
:104100003204982790933204F09234042536310516
:1041100008F4AFCF61E070E08CEC0E94921D81E06A
:104120000E94731D0E94AF1D43C020912E04309148
:104130002F04F901E653FC4F8083909132049827B5
:1041400090933204C901019690932F0480932E041A
:1041500020913004309131048217930708F489CFFD
:104160000093340486CF8091320482130BC0609197
:104170002E0470912F044AEC53E0809133040E9486
:10418000B61D0DC062E070E08BEC0E94921D809124
:1041900033040E94731D809168050E94731DFE0107
:1041A000812F11928A95E9F710922F0410922E0414
:1041B000109234045ECFCDB7DEB7E8E00C94322E17
:1041C00081E08093690580916905882349F080EE3C
:1041D00095E00E94732B892BB1F30E942720F3CF27
:1041E0000895AAE2B0E0E7EFF0E20C94142E0E94EA
:1041F00067286B017C0181E00E947E0A80EE95E0D9
:104200000E94732B892B29F080EE95E00E94A02B51
:10421000F5CF2D9811E072E6B72EE9E2AE2E03E05D
:104220000E9467286C197D098E099F09693C7105F8
:1042300081059105D0F11123C1F10E9467286B011E
:104240007C012C9A80ED97E00E94A807B982E4E7F0
:10425000F5E0DE0112968A2D01900D928A95E1F724
:104260006AE2CE0101960E94DB0B2C9880E090E080
:104270000E94A807009371050E94590B62E370E049
:1042800080E090E00E94962880917105843061F46E
:10429000009371058FE70E9477090E948A0911E057
:1042A000823419F410E001C011E08BE00E948C29E7
:1042B000892B81F411E00EC02D9A2C9A80EE95E0A6
:1042C0000E94A02B8D309105A9F05CF40A9791F023
:1042D0002D982C9880EE95E00E94732B892B61F726
:1042E0009FCF8332910579F08234910589F70E943E
:1042F000E020EECF62EB71E080EE95E00E944D2A67
:104300000E94491DE5CF0E94D215E2CF8F929F9265
:10431000AF92BF92CF92DF92EF92FF921F93CF9313
:10432000DF938BE00E948C29892B09F089C068EC0F
:1043300070E080E090E00E94962880E090E00E948B
:10434000A8070E9467284B015C016B017C0180EC8F
:10435000C80E82E1D81EE11CF11C0E9467286C1572
:104360007D058E059F0530F48BE00E948C29892BFA
:10437000A1F364C08BE00E948C29892B09F05EC0F8
:1043800080ED97E00E94A8070E9467286B017C01DE
:10439000D0E0C1E088E4880E86E2981EA11CB11C22
:1043A00011E08BE00E948C29892B21F58C149D044F
:1043B000AE04BF0430F480ED97E00E94A807D1E07E
:1043C000F0CF0E9467286C197D098E099F09693C0E
:1043D00071058105910528F30E9467286B017C0116
:1043E000C12719F080ED97E002C080E090E00E94C4
:1043F000A807D7CF80E090E00E94A807DD23B9F09E
:104400008091D10590E0019665E070E00E94B72DA3
:104410008093D1050E94290D0E94A9130E94480D86
:1044200064EF71E080E090E00E94962809C080E08F
:104430000E94DF060E94C0110E943F0D0E94F120E1
:10444000DF91CF911F91FF90EF90DF90CF90BF90C1
:10445000AF909F908F900895CF92DF92EF92FF924E
:1044600080E00E94DA070E94B10761E08DE00E94BF
:10447000202961E08CE00E94202960E08BE00E940E
:10448000202960E083E00E94202961E083E00E940F
:10449000592961E08EE00E94202960E08EE00E94B0
:1044A00059290E949F0740E052EC61E070E080EEE5
:1044B00095E00E94BB2C0E94A9130E94480D0E9407
:1044C00092138FEF8093A8040E94C60778940E94ED
:1044D00067286B017C018091A8048F3F59F40E94EA
:1044E00067286C197D098E099F09603D7740810519
:1044F000910588F380ED97E00E94A80761E08BE0CA
:104500000E9459292D9A80EE95E00E94732B892BE9
:1045100029F080EE95E00E94A02BF5CF6DEF72E0C0
:1045200080EE95E00E942E2A82E893E00E94300CF3
:1045300064E173E080EE95E00E942E2A4AE050E0AC
:1045400062E070E080EE95E00E94FE2A62E370E097
:1045500080E090E00E94962880EE95E00E94732B08
:1045600004970CF180EE95E00E94A02B8234910517
:10457000D1F480EE95E00E94A02B8E34910599F441
:1045800080EE95E00E94A02B8434910561F480EECA
:1045900095E00E94A02B819731F480E090E00E948A
:1045A000A8070E94F1204091750550917605609111
:1045B000770570917805DB01CA010197A109B1095E
:1045C0000497A105B10568F44093A704433029F48A
:1045D00040EA56E861E070E004C040E052EC61E07F
:1045E00070E080EE95E00E94BB2C0E9486212D9801
:1045F00080E090E00E94A8070E9492131092C304EA
:104600008091BD0583FF11C080918905882351F0F9
:1046100080919005882331F080919705882311F0CF
:1046200087E001C085E08093C30480E00E947E0A99
:104630008091C4040E94B2090E94590B10923F0459
:1046400010923E0410923D04F12C8091D2058F15FA
:10465000B0F062E370E080E090E00E94962880ED88
:1046600097E00E94A80762E370E080E090E00E947B
:10467000962880E090E00E94A807F394E6CF80910E
:104680009C0584FF08C0982F987181E0983109F04B
:1046900080E00E947C118FE00E94DA07FF90EF908B
:1046A000DF90CF900895EF92FF920F931F93CF93D7
:1046B000DF938C016EE770E080EE95E00E94590672
:1046C000E801F12CF0E2EF2E8E0188818D578230C7
:1046D00048F46DE770E080EE95E00E94590688810D
:1046E0008E2588832196F801608180EE95E00E94F6
:1046F000CD2BF394F9E0FF12E7CF6EE770E080EE88
:1047000095E00E945906CDB7DEB7E6E00C94342E52
:10471000A9E0B0E0EEE8F3E20C941C2E9091C50401
:1047200091110EC09EEF99838A836B8350E055955B
:1047300047954C832D83198618861F821E822EC0B2
:104740004091CA04842F90E0B4E095958795BA957E
:10475000E1F7242F2F7030E08217930719F18DEFC6
:1047600089831B82FE01349650E0842F90E0A4E000
:1047700095958795AA95E1F7242F2F7030E0821741
:10478000930749F0DC01A553BB4F8C918193405FA7
:104790005F5F563051F74093CA045A83CE010196A9
:1047A0000E9453238091C50490E0019666E070E07A
:1047B0000E94B72D8093C5042996E2E00C94382E10
:1047C000A0E0B0E0E6EEF3E20C94152E6C016EE78B
:1047D00070E080EE95E00E9459068601E12CF12CF4
:1047E000C0E0D0E030E2B32EF801608183E8860FAC
:1047F000823078F46DE770E080EE95E00E94590613
:10480000F80160816B2570E080EE95E00E9459060A
:1048100004C080EE95E00E94CD2BE114F10459F024
:10482000F80180819E01280F311DC901C92FDD27A4
:10483000C80FD91FDD273FEFE31AF30A89E0E81616
:10484000F10459F028E0E216F10421F48C2F809550
:10485000F60180870F5F1F4FC7CFCDB7DEB7E9E006
:104860000C94312EA9E0B0E0E8E3F4E20C941C2EA5
:10487000E82F362F8091C50490E0019664E270E045
:104880000E94B72D8093C50458E9598350E15A839B
:10489000813089F048F08230B9F08330D9F48B83CD
:1048A00081EF8C833D8319C085E08B8381EF8C83FE
:1048B0002F5F2D8312C08B8381EF8C8384E6489F0A
:1048C000A00111245D8309C084E08B8381EF8C8378
:1048D000ED8303C00E94B91104C0CE0101960E946D
:1048E000E0232996E2E00C94382EA2E0B0E0EBE75A
:1048F000F4E20C94112E182F762E2A8349830E94FD
:1049000073286B017C018091DB048090C604909039
:10491000C704A090C804B090C9042A8149818823A3
:10492000C1F0D701C60188199909AA09BB094C0130
:104930005D0191EE89169EE29906A104B10420F171
:10494000241708F4422F202F672D812F0E94322434
:1049500013C0D701C60188199909AA09BB094C01DE
:104960005D0191E3891695E79906A104B10460F011
:10497000672D812F0E948823C092C604D092C7045D
:10498000E092C804F092C9042296EDE00C942D2E1A
:10499000A2E2B0E0EEECF4E20C94122E8CE00E9465
:1049A000990981110DC06CE173E080EE95E00E94E1
:1049B0005F2A2D9A80E00E947E0A0E94590B2D9852
:1049C00080EE95E00E94732B892B01F180EE95E03B
:1049D0000E94A02B9091A704992319F00E94BC1368
:1049E000EFCF40913E0450E09A012F5F3F4F2F716F
:1049F000332760913F0470E02617370709F3FA0167
:104A0000E75BFB4F808320933E04DACF80917105F2
:104A1000843009F086C00E947328611571058105F4
:104A2000910549F06093B5047093B6048093B70480
:104A30009093B8040CC081E090E0A0E0B0E08093D7
:104A4000B5049093B604A093B704B093B8048091D2
:104A5000AB049091AC0481609093AC048093AB0460
:104A600083E0809371058FE70E94770909E614E0DF
:104A70000E948A09F80181938F01F4E002371F0731
:104A8000B9F72091720480916904982F922796FFBC
:104A90003BC090E4922790937204982F98739833B8
:104AA000F1F410E0212F30E080916904877090E0EC
:104AB000821793074CF11F5F20919C05812F90E096
:104AC000FC01E759FB4F24FF04C080810E949B1129
:104AD000E9CF608180EE95E00E94CD2BE3CF8F730C
:104AE00099F480916A048093B40480916B0480935C
:104AF000B20480916C048093B10480916F0490E0C3
:104B00009093AA048093A90480913D04813019F404
:104B100082E080933D0480913D04833011F4109233
:104B20003D040E9473286B017C018091AD0490913B
:104B3000AE04A091AF04B091B0040097A105B105F7
:104B4000C9F0A7019601281B390B4A0B5B0BDA0150
:104B5000C901883B9B40A105B10560F00E94C809CE
:104B60008093B3041092AD041092AE041092AF047F
:104B70001092B0048091B9049091BA04A091BB0442
:104B8000B091BC0446015701881A990AAA0ABB0AC7
:104B900084E795E00E94F40786169706A806B906F2
:104BA00008F4A8C0C092B904D092BA04E092BB0441
:104BB000F092BC040E9457068091A8048830A0F0AF
:104BC0008091BD059091BE05A091BF05B091C00533
:104BD0005CE1B695A795979587955A95D1F7892B5E
:104BE0008A2B8B2B09F09EC18091A8048F5F809344
:104BF000A8048091B5049091B604A091B704B09137
:104C0000B8040097A105B105F1F0C81AD90AEA0A5B
:104C1000FB0A84E795E00E94F4076C157D058E057C
:104C20009F0508F006C18091BD0584FD04C080ED9C
:104C300097E00E94A8071092B5041092B604109253
:104C4000B7041092B80490917204907C909372040F
:104C500050913E0480913F0420913D04581709F47F
:104C600005C1223009F002C1905890937204E0917E
:104C70009C05E770F0E0E658FC4F6081693008F071
:104C8000DDC0615040E04613DBC080933F0487E302
:104C9000840F90917204892B809372044093400496
:104CA00083E080933D042C9A809181059091C30408
:104CB000911129C10E94790A8091C4040E94B2090D
:104CC000E0919C05E770F0E0E658FC4F608182E7D8
:104CD00094E00E94940BE091C404EF5FE093C4045D
:104CE000E83109F41CC1F0E0EC58FA4F87858823BD
:104CF00009F415C10E94030C813069F580919C056F
:104D0000887149F18091AB049091AC04880F991F90
:104D10009093AC048093AB0483E0809371050E9470
:104D2000590B0E9473286093AD047093AE04809376
:104D3000AF049093B004672B682B692B61F481E07A
:104D400090E0A0E0B0E08093AD049093AE04A09317
:104D5000AF04B093B00480919C0584FF1FC0809184
:104D6000AB049091AC048E7F0E942A09182F6091A9
:104D7000A9048091B4040E94B213482F612F80913E
:104D8000B30449A30E94B2130091D205282F49A170
:104D90006091B1048091B2040E9475242C98809196
:104DA000C1048130C1F018F08230B1F1C8C08BE08D
:104DB0000E948C29892B09F0C2C081E08093C10434
:104DC0000E9467286093BD047093BE048093BF0463
:104DD0009093C004B4C08BE00E948C29892B31F5DC
:104DE0000E946728C090BD04D090BE04E090BF042C
:104DF000F090C0046C197D098E099F09693E7340CB
:104E00008105910508F49BC082E08093C10480ED88
:104E100097E00E94A80793C08BE00E948C29892B01
:104E200009F48DC080E090E00E94A8071092C104B0
:104E300086C080E090E00E94A80705CF68E022CFFE
:104E4000851709F422CF4F5F242F30E090E0F9015D
:104E5000EE58FB4FDC01A75BBB4F7C917083F901DF
:104E6000E05CFB4F708301968F710DCF2430B1F45D
:104E70002091400481E494E0A3E7B4E0FC013E2FDC
:104E8000381B321718F431913D93F9CF87E3820F25
:104E900090917204892B8093720402CF8091C10497
:104EA000823051F49160909372042D9A8E010F5FBD
:104EB0001F4FF12CB80110C02D9880913D04811135
:104EC00003C081E080933D0480913D04833071F7FD
:104ED00084E080933D04EACF8F2D69A37AA30E94DA
:104EE000B415F801819391938F01F39469A17AA18C
:104EF000F0E1FF12F1CF80919C0543E754E0877009
:104F00000E947908D0CE882309F4D4CE2091C2041F
:104F100031E0320F3093C2042913CCCE0CC0109272
:104F2000C404E8CE8091A804883009F42D9A89E061
:104F30008093A804DFCE1092C2048150BBCEA2960B
:104F4000ECE00C942E2E8230E8F4E82FF0E0EE0F27
:104F5000FF1FED52FA4F71836083813041F08091E1
:104F600069008C7F842B80936900E89A0895809172
:104F70006900440F551F440F551F837F842B809376
:104F80006900E99A08951F920F920FB60F921124AB
:104F90002F933F934F935F936F937F938F939F9341
:104FA000AF93BF93EF93FF938091D3059091D40576
:104FB000892B29F0E091D305F091D4050995FF9153
:104FC000EF91BF91AF919F918F917F916F915F9181
:104FD0004F913F912F910F900FBE0F901F901895FA
:104FE0001F920F920FB60F9211242F933F934F935E
:104FF0005F936F937F938F939F93AF93BF93EF9341
:10500000FF938091D5059091D605892B29F0E091E9
:10501000D505F091D6050995FF91EF91BF91AF911C
:105020009F918F917F916F915F914F913F912F91C0
:105030000F900FBE0F901F9018951F920F920FB6F2
:105040000F9211242F933F938F939F93AF93BF930E
:105050008091D8059091D905A091DA05B091DB0532
:105060003091D70523E0230F2D3720F40196A11DA1
:10507000B11D05C026E8230F0296A11DB11D209386
:10508000D7058093D8059093D905A093DA05B093FE
:10509000DB058091DC059091DD05A091DE05B091E6
:1050A000DF050196A11DB11D8093DC059093DD0500
:1050B000A093DE05B093DF05BF91AF919F918F91D3
:1050C0003F912F910F900FBE0F901F9018952FB703
:1050D000F8946091D8057091D9058091DA05909186
:1050E000DB052FBF08953FB7F8948091DC059091C0
:1050F000DD05A091DE05B091DF0526B5A89B05C0B2
:105100002F3F19F00196A11DB11D3FBF6627782FD3
:10511000892F9A2F620F711D811D911D42E0660F2C
:10512000771F881F991F4A95D1F70895CF92DF9274
:10513000EF92FF92CF93DF936B017C010E94732863
:10514000EB01C114D104E104F10479F00E94732849
:105150006C1B7D0B683E7340A0F381E0C81AD10838
:10516000E108F108C851DC4FECCFDF91CF91FF90FF
:10517000EF90DF90CF900895789484B5826084BDDD
:1051800084B5816084BD85B5826085BD85B581604B
:1051900085BDEEE6F0E0808181608083E1E8F0E0AB
:1051A0001082808182608083808181608083E0E8DA
:1051B000F0E0808181608083E1EBF0E080818460B9
:1051C0008083E0EBF0E0808181608083EAE7F0E0BB
:1051D000808184608083808182608083808181601F
:1051E00080838081806880831092C100089583301D
:1051F00081F028F4813099F08230A1F00895863052
:10520000A9F08730B9F08430D1F4809180008F7D8F
:1052100003C0809180008F7780938000089584B5CB
:105220008F7702C084B58F7D84BD08958091B000D2
:105230008F7703C08091B0008F7D8093B000089578
:10524000CF93DF9390E0FC01ED50F44F2491FC01EB
:10525000E95FF34F8491882349F190E0880F991F0B
:10526000FC01E15DF34FA591B4918B5D934FFC017F
:10527000C591D4919FB7611108C0F8948C91209585
:1052800082238C93888182230AC0623051F4F8947F
:105290008C91322F309583238C938881822B888345
:1052A00004C0F8948C91822B8C939FBFDF91CF9197
:1052B0000895A1E0B0E0EFE5F9E20C941A2E282F52
:1052C00030E0F901E152F44F8491F901ED50F44FCF
:1052D0001491F901E95FF34F04910023C9F0882389
:1052E00021F069830E94F7286981E02FF0E0EE0F3A
:1052F000FF1FEB5DF34FA591B4919FB7F8948C918C
:10530000611103C01095812301C0812B8C939FBF35
:105310002196E4E00C94362ECF93DF93282F30E0D3
:10532000F901E152F44F8491F901ED50F44FD49119
:10533000F901E95FF34FC491CC2391F081110E94F0
:10534000F728EC2FF0E0EE0FFF1FE55EF34FA5917D
:10535000B4912C912D2381E090E021F480E002C0F3
:1053600080E090E0DF91CF9108958E3008F08E506C
:10537000877020919D0190E4299F90011124822B38
:1053800080937C0080917A00806480937A00809181
:105390007A0086FDFCCF809178002091790090E022
:1053A000922B0895A0E0B0E0E8EDF9E20C94162EFF
:1053B0006C017A01EB01E60EF71E00E010E0CE155D
:1053C000DF0561F06991D601ED91FC910190F081CA
:1053D000E02DC6010995080F191FF1CFC801CDB7FF
:1053E000DEB7E8E00C94322E6115710589F0DB011F
:1053F0000D900020E9F7AD0141505109461B570BB4
:10540000DC01ED91FC910280F381E02D0995089576
:1054100080E090E00895EF92FF920F931F93CF9357
:10542000DF938C01FB01C0E0D0E064917F018FEF3E
:10543000E81AF80A662361F0D801ED91FC91019019
:10544000F081E02DC8010995C80FD91FF701EDCFF4
:10545000CE01CDB7DEB7E6E00C94342E0E94F429DD
:105460000895DC01ED91FC910190F081E02D09950A
:1054700008950F931F93CF93DF93EC016DE00E948B
:10548000312A8C016AE0CE010E94312A800F911FDF
:10549000DF91CF911F910F9108950F931F93CF9399
:1054A000DF93EC010E940B2A8C01CE010E94392A65
:1054B000800F911FDF91CF911F910F9108950F934E
:1054C0001F93CF93DF93EC010E94F4298C01CE014E
:1054D0000E94392A800F911FDF91CF911F910F9168
:1054E00008950F931F93CF93DF93EC010E94312A0D
:1054F0008C01CE010E94392A800F911FDF91CF913C
:105500001F910F910895A1E2B0E0E9E8FAE20C944E
:10551000122E7C01C42EE52FCB01D22E19A221E040
:105520002D1510F02AE0D22E8E010F5D1F4F8D2C0D
:10553000912CA12CB12C6C2D7E2FA50194010E94E1
:10554000CB2D8C2DD29E80191124015011098A3047
:1055500010F4805D01C0895CF8018083211531055C
:105560004105510521F0C22EE32FCA01E4CFB80155
:10557000C7010E94F429A196ECE00C942E2EA0E025
:10558000B0E0E5ECFAE20C94162EEC016A017B0126
:105590002115310541F4E881F9810190F081E02D78
:1055A000642F09951DC02A303105A9F477FF12C078
:1055B0006DE20E94312A8C0144275527BA014C190B
:1055C0005D096E097F092AE0CE010E94832A800FBF
:1055D000911F06C02AE0B701A601CE010E94832ACE
:1055E000CDB7DEB7E8E00C94322E9A01AB01662706
:1055F00057FD6095762F0E94BF2A08950F931F9341
:10560000CF93DF93EC019A01AB01662757FD6095BC
:10561000762F0E94BF2A8C01CE010E94392A800F6A
:10562000911FDF91CF911F910F91089521153105A1
:1056300049F4DC01ED91FC910190F081E02D642FA3
:10564000099508950E94832A08959A01462F50E0F3
:1056500060E070E00E94162B08959A01AB0160E0B3
:1056600070E00E94162B08950F931F93CF93DF9342
:10567000EC010E94162B8C01CE010E94392A800F6A
:10568000911FDF91CF911F910F9108950F931F9359
:10569000CF93DF93EC019A01AB0160E070E00E94D0
:1056A000162B8C01CE010E94392A800F911FDF91A9
:1056B000CF911F910F9108950F931F93CF93DF9375
:1056C000EC019A01462F50E060E070E00E94162B3A
:1056D0008C01CE010E94392A800F911FDF91CF915A
:1056E0001F910F910895FC0124853585F901E05C37
:1056F000FF4F80819181F901EE5BFF4F2081318165
:10570000821B930B8F7399270895FC0184859585DF
:10571000FC01E05CFF4F40815181FC01EE5BFF4FDB
:10572000208131814217530741F00190F081E02D33
:10573000E80FF91F808190E008958FEF9FEF0895A3
:10574000FC0184859585FC01E05CFF4F408151811F
:10575000FC01EE5BFF4F208131814217530779F046
:10576000A081B181A80FB91F8C91208131812F5F59
:105770003F4F2F7333273183208390E008958FEFBD
:105780009FEF0895FC0181A1882329F0A489B589A0
:105790008C9186FFFBCF11A20895CF93DF93FC017C
:1057A00026853785D901A05CBF4F8D919C911197BB
:1057B00001968F739927E901CE5BDF4F48815981AC
:1057C00084179507D9F30D90BC91A02DA20FB31F9C
:1057D0006C93A685B785A05CBF4F11969C938E9362
:1057E000A689B7892C9181E090E0078C02C0880FD0
:1057F000991F0A94E2F7282B2C9381E081A3048857
:10580000F589E02D80818064808381E090E0DF91E4
:10581000CF91089508951F920F920FB60F92112401
:105820002F933F934F938F939F93EF93FF93809189
:10583000C00082FD1CC04091C600809186069091F8
:10584000870601968F7399272091880630918906E3
:105850008217930771F0E0918606F0918706EA5B64
:10586000F94F4083909387068093860602C080910B
:10587000C600FF91EF919F918F914F913F912F9192
:105880000F900FBE0F901F90189580EE95E00E942C
:10589000732B892B11F00E940A2C08951F920F92EE
:1058A0000FB60F9211242F933F938F939F93EF93F3
:1058B000FF932091420630914306809144069091D7
:1058C00045062817390731F48091C1008F7D8093F8
:1058D000C10014C0E0914406F0914506EE5FF94F17
:1058E0002081809144069091450601968F739927F7
:1058F00090934506809344062093C600FF91EF9154
:105900009F918F913F912F910F900FBE0F901F90FD
:105910001895A0E0B0E0EFE8FCE20C94122EFC0138
:105920001382128288EE93E0A0E0B0E08483958336
:10593000A683B7838CEB93E091838083758764871C
:1059400057874687318B208B138B028BF58AE48A2D
:10595000D78AC68AB18EA08E938E828E8F85848FD1
:105960008889858F8989868F8A89878F8B8980A38B
:10597000ECE00C942E2ECF92DF92EF92FF92CF9319
:10598000DF93EC016A017B01411581EE5807610547
:105990007105F9F0EC89FD8981E090E008A002C072
:1059A000880F991F0A94E2F7808360E079E08DE325
:1059B00090E0A70196010E94CB2D215031094109A9
:1059C00051095695479537952795211580E1380758
:1059D00098F0EC89FD89108260E874E88EE190E02F
:1059E000A70196010E94CB2D21503109410951098F
:1059F0005695479537952795E889F9893083EA893F
:105A0000FB89208319A2EE89FF89408181E090E023
:105A10009C010C8C02C0220F331F0A94E2F7422B28
:105A20004083EE89FF8940819C010D8C02C0220FCA
:105A3000331F0A94E2F7422B4083EE89FF894081AD
:105A40009C010E8C02C0220F331F0A94E2F7422BF6
:105A50004083EE89FF8920810F8C02C0880F991F37
:105A60000A94E2F7809582238083DF91CF91FF90A3
:105A7000EF90DF90CF9008958F929F92AF92BF9258
:105A8000CF92DF92EF92FF920F931F9381E08F935B
:105A900085E08F9387E08F9383E08F9384E08F93EB
:105AA000E6EC8E2E912CF2ECAF2EB12CA1ECCA2E8E
:105AB000D12CB0ECEB2EF12C04EC10E025EC30E016
:105AC00042E056E066E476E080EE95E00E94892CA4
:105AD0000F900F900F900F900F901F910F91FF90CC
:105AE000EF90DF90CF90BF90AF909F908F900895F0
:105AF0000E94BC280E942C22C5E4DCE20E94C8243B
:105B00002097E1F30E94452CF9CFA29FB001B39FEB
:105B1000C001A39F700D811D1124911DB29F700DB6
:105B2000811D1124911D08950E94852DA59F900D22
:105B3000B49F900DA49F800D911D11240895B7FF6F
:105B40000C94942D0E94942D821B930B0895DB01DD
:105B50008F939F930E94942DBF91AF91A29F800D30
:105B6000911DA39F900DB29F900D1124089597FB56
:105B7000072E16F4009407D077FD09D00E94492E15
:105B800007FC05D03EF4909581959F4F0895709540
:105B900061957F4F0895A1E21A2EAA1BBB1BFD0140
:105BA0000DC0AA1FBB1FEE1FFF1FA217B307E407FC
:105BB000F50720F0A21BB30BE40BF50B661F771F54
:105BC000881F991F1A9469F7609570958095909534
:105BD0009B01AC01BD01CF010895052E97FB1EF47A
:105BE00000940E94042E57FD07D00E94CB2D07FC85
:105BF00003D04EF40C94042E509540953095219589
:105C00003F4F4F4F5F4F08959095809570956195E8
:105C10007F4F8F4F9F4F08952F923F924F925F92E9
:105C20006F927F928F929F92AF92BF92CF92DF92AC
:105C3000EF92FF920F931F93CF93DF93CDB7DEB711
:105C4000CA1BDB0B0FB6F894DEBF0FBECDBF0994A5
:105C50002A88398848885F846E847D848C849B84FC
:105C6000AA84B984C884DF80EE80FD800C811B810A
:105C7000AA81B981CE0FD11D0FB6F894DEBF0FBE39
:105C8000CDBFED010895EE0FFF1F0590F491E02DBB
:105C90000994AA1BBB1B51E107C0AA1FBB1FA61773
:105CA000B70710F0A61BB70B881F991F5A95A9F7C5
:105CB00080959095BC01CD0108958F929F92AF92EF
:105CC000BF92CF92DF92EF92FF92CF93DF93EC01DE
:105CD000688179818A819B816115710581059105B2
:105CE00021F464E279ED8BE597E02DE133EF41E0BB
:105CF00050E00E94ED2D49015A019B01AC01A7EA39
:105D0000B1E40E94942D6B017C01ACEEB4EFA501CF
:105D100094010E94A22DC60ED71EE81EF91EF7FEA2
:105D200006C081E0C81AD108E10880E8F80AC882F4
:105D3000D982EA82FB82C701B6019F77DF91CF91BA
:105D4000FF90EF90DF90CF90BF90AF909F908F909B
:105D500008950E945D2E089586E091E00E945D2ED8
:105D60000895609306017093070180930801909352
:105D7000090108952F923F925F926F927F928F92C6
:105D80009F92AF92BF92CF92DF92EF92FF920F93CA
:105D90001F93CF93DF938B01EA016115710521F009
:105DA000DB018C9311969C93209739F09E01225031
:105DB00031092332310508F0D8C07C016701BFEFFB
:105DC000CB1ADB0A5601F7016080862D90E00E9415
:105DD000EC2F892B11F07601F1CFFDE26F120AC092
:105DE000570182E0A80EB11CD70111966C90772460
:105DF00073940BC0BBE26B1207C05701E2E0AE0E1A
:105E0000B11CD70111966C90712CCE018F7E892B1D
:105E100089F4B0E36B1237C0F50180818F7D88353E
:105E2000D1F46180F2E0AF0EB11C872D8260782E34
:105E3000C0E1D0E0CA30D10551F1C031D10521F027
:105E4000C830D10599F409C0CC24CA94DC2CEC2CC0
:105E5000AFE0FA2E22C0209769F7C8E0D0E0CC244A
:105E6000CA94DC2CEC2CFFE1FF2E17C06FEF7FEF04
:105E7000CB019E01442737FD4095542F0E94CB2D26
:105E800069017A010AC02097A9F6CAE0D0E0E9E9E1
:105E9000CE2EDC2CEC2CE9E1FE2EF50160E020E0BA
:105EA00030E0A9014E01AA2497FCA094BA2C1F014E
:105EB00070ED572E560CA9E0A51570F48FEB860DEA
:105EC0008A3118F499EC592E06C08FE9860D8A3173
:105ED00048F589EA582E560C852D90E08C179D07C1
:105EE0000CF56F3FD9F0C216D306E406F50698F01C
:105EF000C501B4010E94A72D9B01AC01852D90E046
:105F0000A0E0B0E0280F391F4A1F5B1F2817390790
:105F10004A075B0710F46FEF01C061E03196D101D1
:105F20006C90C5CF0115110551F0662311F0319722
:105F300003C071FE04C03297D801ED93FC9370FE4C
:105F400007C050954095309521953F4F4F4F5F4F7B
:105F500067FF10C082E290E090938B0680938A06E0
:105F60006FEF7FEF8FEF9FEF07C060E070E080E0A2
:105F700090E002C0B901CA01DF91CF911F910F914A
:105F8000FF90EF90DF90CF90BF90AF909F908F9059
:105F90007F906F905F903F902F900895FC0188272D
:105FA0009927E89421912032E9F3293010F02E301E
:105FB000C8F32B3241F02D3239F4689404C00E94AA
:105FC0002030820F911D219120532A30C0F31EF4FE
:105FD000909581959F4F0895911150C0803219F08E
:105FE00089508550D0F7089548EC53E00E94F92F6E
:105FF0000895FA01A191B081009719F41097E1F08A
:10600000CD01DC01CD010D90002011F4C00113C0C1
:10601000FB012191222319F02015D9F7F3CFFB01C1
:106020002191201519F41E92119606C02223C1F762
:106030000D900020A1F7D001FA01A193B08308953B
:106040007AE0979F902D879F802D910D11240895C0
:10605000F999FECF92BD81BDF89A992780B5089530
:10606000262FF999FECF1FBA92BD81BD20BD0FB674
:10607000F894FA9AF99A0FBE0196089599278827FD
:066080000895F894FFCF23
:1060860000008C06200001000000FF000200020054
:1060960002000200020002000200020002000200EA
:1060A6000200020002000200020002802500000534
:1060B600400AA1204EA50020244EA52C2330C01254
:1060C60000001A400AA1204EA5001B1E27522C23B1
:1060D600308025000005400AA1204EA50020244E50
:1060E600A52C2330004B000006400AD0009D490035
:1060F6007B289D492C233000E1000005400A45011C
:10610600D7DC03B81E0EBF00232E48E801008A40E4
:106116000A6001555502AD1E20000023C8015458DF
:106126002074696D656F75742100596573004E6F33
:10613600002C00386368004E2F41002C205B005D68
:106146002028002900486F70206368616E6E656CB8
:10615600200020402000456E746572696E672061DC
:1061660064617074697665206368616E6E656C2023
:1061760073656C656374696F6E2C207069636B69F7
:106186006E673A007363616E6E6572206D6F64654B
:10619600004E4F5420454E41424C45440053656ED7
:1061A60064696E672073657474696E677320746FB3
:1061B6002052580A00526573657474696E672073BD
:1061C600657474696E6773206F6E2052580A0041B9
:1061D600626F727465642065646974730A00696E1F
:1061E60076616C69642073656C656374696F6E00B3
:1061F6000D0A496E76616C696420696E707574204B
:106206002D206469736361726465642107005365B8
:106216007474696E677320736176656420746F2089
:10622600454550524F4D0A00526576657274656455
:106236002073657474696E67732066726F6D20458E
:106246004550524F4D0A004C6F616465642066618B
:1062560063746F72792064656661756C74730A0085
:106266004B657920616E64206368616E6E656C7340
:106276002072616E646F6D697A65640A004F70659D
:106286006E4C52536E672054582073746172746951
:106296006E672000206F6E20485720006D6F647572
:1062A6006C65206C6F636B65643F00342B3400387B
:1062B60000382B340031320031322B3400313600B5
:1062C60050504D0052535349005344410053434CE0
:1062D60000525844005458440041494E004C42452F
:1062E60045500053504B54524D00534255530053A2
:1062F600554D44004C4C494E440000070B0C101100
:106306001500B7012B032F033103350338033D0373
:10631600B7014003440349034D0351035503590391
:106326005D0363036A036F0374038D028D028D029E
:106336008D02160A1322312900000000CD2BD22926
:08634600732BA02B852BC22B49
:00000001FF
